:0A1E9E00000102020303040405051D
:10068300E4F513F512F511F510C203C200C202C25C
:1006930001121D961209BF7E147F008E528F53756F
:1006A3005A14755B1275501475511C75581475598D
:1006B3004A755C14755D78EE54E070030207CA75E1
:1006C30014007515808E168F17C374A29FFF7414C0
:1006D3009ECF2402CF3400FEE48F0F8E0EF50DF56E
:1006E3000CF50BF50AF509F508AF0FAE0EAD0DAC21
:1006F3000CAB0BAA0AA909A808C31209AE5026E538
:1007030015250BF582E514350AF58374CDF0E50B59
:100713002401F50BE4350AF50AE43509F509E43556
:1007230008F50880C4E4F50BF50AF509F508AF0FE1
:10073300AE0EAD0DAC0CAB0BAA0AA909A808C312E7
:1007430009AE5031AE0AAF0BE5172FF582E5163E21
:10075300F583E0FDE5152FF582E5143EF583EDF015
:10076300EF2401F50BE43EF50AE43509F509E43518
:1007730008F50880B985145285155374002480FF49
:10078300741434FFFEC3E55B9FF55BE55A9EF55A8F
:10079300C3E5559FF555E5549EF554C3E5579FF5BD
:1007A30057E5569EF556C3E5519FF551E5509EF525
:1007B30050C3E5599FF559E5589EF558C3E55D9F2C
:1007C300F55DE55C9EF55CD2E843D82090E668E0F1
:1007D3004409F090E65CE0443DF0D2AF90E680E05F
:1007E30020E105D208121BDD90E680E054F7F053B8
:1007F3008EF8C20330010512045FC20130032912CF
:100803001F2C5024C203121D3520001690E682E0EF
:1008130030E704E020E1EF90E682E030E604E020F8
:0D082300E0E4121C0C121F2E1214A480C75A
:10045F0090E6B9E0700302051014700302058D24B5
:10046F00FE700302061024FB700302050A147003CA
:10047F000205041460731460762405600302066F8E
:10048F00121F30400302067B90E6BBE024FE602281
:10049F0014603324FD601114602224067048E55265
:1004AF0090E6B3F0E5538037E55A90E6B3F0E55B9D
:1004BF00802DE55490E6B3F0E5558023E55690E6A0
:1004CF00B3F0E557801990E6BAE0FF121C38AA0680
:1004DF00A9077B01EA494B600DEE90E6B3F0EF9070
:1004EF00E6B4F002067B020674121E4702067B1268
:1004FF001F0E02067B121A2F02067B121E350206F2
:10050F007B121F32400302067B90E6B8E0247F6027
:10051F001514601924027063A200E43325E0FFA2D2
:10052F0002E4334F8041E490E740F0803F90E6BC17
:10053F00E0547EFF7E00E0D394807C0040047D0178
:10054F0080027D00EC4EFEED4F249EF582741E3E20
:10055F00F583E493FF3395E0FEEF24A1FFEE34E63D
:10056F008F82F583E0540190E740F0E4A3F090E62A
:10057F008AF090E68B7402F002067B020674121F5B
:10058F0034400302067B90E6B8E024FE6016240296
:10059F00600302067B90E6BAE0B40105C2000206D2
:1005AF007B02067490E6BAE0705590E6BCE0547E8C
:1005BF00FF7E00E0D394807C0040047D0180027DAB
:1005CF0000EC4EFEED4F249EF582741E3EF583E443
:1005DF0093FF3395E0FEEF24A1FFEE34E68F82F513
:1005EF0083E054FEF090E6BCE05480131313541FC5
:1005FF00FFE0540F2F90E683F0E04420F0806D80F1
:10060F0064121F36506690E6B8E024FE601924028B
:10061F00705A90E6BAE0B40104D200804F90E6BA67
:10062F00E064026047803E90E6BCE0547EFF7E00AF
:10063F00E0D394807C0040047D0180027D00EC4E6D
:10064F00FEED4F249EF582741E3EF583E493FF3337
:10065F0095E0FEEF24A1FFEE34E68F82F58380084C
:10066F00120080500790E6A0E04401F090E6A0E071
:03067F004480F0C4
:010682002255
:03003300021F2584
:041F250053D8EF326C
:101D9600758CE0758AC0E58954F04401F589758E25
:081DA60003D28CD2A9D2AF22B6
:03000B0002116778
:10116700C0E0C0F0C083C082C0D075D000C000C04E
:1011770001C002C003C004C005C006C007758CE0EB
:10118700758AC0D28CE47F607EEAFDFCAB4FAA4E25
:10119700A94DA84CC31209AE5019AF4FAE4EAD4D75
:1011A700AC4CEF2401F54FE43EF54EE43DF54DE43C
:1011B7003CF54CE47F01FEFDFCAB4FAA4EA94DA8C0
:1011C7004CC31209AE7008E5A054F02534F5A0E52C
:1011D7002B2401FFE4352AFEE4FCFDAB4FAA4EA900
:1011E7004DA84CC31209AE700553A0F0C28CD007AE
:1011F700D006D005D004D003D002D001D000D0D083
:09120700D082D083D0F0D0E03297
:101400001201000200000040181601120000010243
:1014100000010A06000200000040010009022E003F
:1014200001010080FA0904000004FF000000070524
:1014300001024000000705820200020007050202C7
:101440000002000705810240000009022E00010190
:101450000080FA0904000004FF00000007050102F3
:10146000400000070582024000000705020200025A
:101470000007058102400000040309041003510025
:10148000480059002D00430043004400160351005A
:10149000480059002D0031003200200020002000BB
:0414A0002000000028
:100CC6006080270002020202020202070000000200
:100CD600000002001332120A080C0800000000008F
:100CE6000000003F020202020202020700000002A8
:100CF600000000002020202000000000000000006E
:100D06000000003F033A0303030303070000000249
:100D1600000002001332120A080C0800000000004E
:100D26000000003F03FAFA03030303070000000272
:100D3600000000002020202000000000000000002D
:100D46000000003F6024278700000000000000002C
:100D5600000000000000000000000000000000008D
:100D6600000000000000000000000000472780800F
:060D7600000000CA4E005F
:100F160090E60174CAF090E6F574FFF0902780E041
:100F260090E6F3F0902781E090E6C3F0902782E008
:100F360090E6C1F0902783E090E6C2F0902785E026
:100F460090E6C0F0902786E090E6F4F075AF07745F
:100F560027F59A7400F59B759DE4E4F59EFF90E6EF
:100F66007BE090E67CF00FBF80F490E67174FFF0B2
:100F7600F5B490E672E04480F043B680000000E4E9
:100F860090E6C4F000000090E6C5F0902787E09058
:100F9600E6C6F0902788E090E6C7F0902789E090B3
:100FA600E6C8F090278AE090E6C9F090278BE0909B
:100FB600E6CAF090278CE090E6CBF090278DE09083
:0B0FC600E6CCF090278EE090E6CDF026
:010FD10022FD
:03004300021000A8
:0300530002100098
:10100000021DAE00021DF400021DDE00021DC6001E
:10101000021AA900021A6C00020FFF00021F38001A
:10102000021F3900021F3A000217E30002135A00A0
:10103000021F3B00021F3C00021F3D00021F3E003A
:10104000021F3F00021F3800021F4000021F410024
:10105000021F4200021F4300021F4400021F4500FE
:10106000021F4600021F3800021F3800021F38000E
:10107000021F4700021F4800021F4900021F4A00CA
:10108000021F4B00021F4C00021F4D00021F4E00AA
:10109000021F4F00021F5000021F5100021F52008A
:1010A000021F5300021F5400021F5500021F56006A
:0810B000021F5700021F580047
:101C0C0090E682E030E004E020E60B90E682E030E3
:101C1C00E119E030E71590E680E04401F07F147E96
:0C1C2C00001218DF90E680E054FEF02269
:101D350090E682E044C0F090E681F0438701000020
:041D45000000002278
:101BDD0030080990E680E0440AF0800790E680E046
:101BED004408F07FDC7E051218DF90E65D74FFF08F
:0F1BFD0090E65FF05391EF90E680E054F7F0220E
:021C3800A907FA
:101C3A00AE5CAF5D8F828E83A3E064037017AD0143
:101C4A0019ED7001228F828E83E07C002FFDEC3E1D
:091C5A00FEAF0580DF7E007F0073
:011C6300225E
:1018DF008E1C8F1D90E600E054187012E51D240138
:1018EF00FFE4351CC313F51CEF13F51D801590E6AF
:1018FF0000E05418FFBF100BE51D25E0F51DE51C9A
:10190F0033F51CE51D151DAE1C7002151C4E600530
:06191F00121D4980EE22BA
:101D49007400F58690FDA57C05A3E582458370F9AD
:011D59002267
:100D7C00C1850223000002311040C1070448000065
:020D8C00000065
:081CBA0090E679F07F057E0041
:101CC2008E1E8F1FE51F451E60177F957E00120E28
:101CD200FF000000000000E51F151F70E7151E80C1
:021CE200E322FB
:1009BF0090E600E054E74410F000000000000090C3
:1009CF00E61074A0F000000090E60B7401F090E6C2
:1009DF001274E0F0000000E490E613F000000090C5
:1009EF00E61474E0F0000000E490E615F00000005B
:1009FF0090E618740CF000000090E6D27402F090AC
:100A0F00E6047480F00000007402F0000000E4F0CF
:100A1F0000000090E61474E0F0000000120F16E4DE
:100A2F0090E671F075B4FF90E672F075B6FF75B190
:100A3F00FF90E670F075B2FFC28CD287D285121E7E
:100A4F007B75230275240000000090E61074A0F05F
:100A5F0000000000000090E611F000000090E65E3C
:100A6F00E04408F0000000E490E68DF090E65EE0D0
:100A7F004404F0000000E490E68FF0121C8F5380C6
:100A8F00FE7F9A7E00121EC67528007529B4754325
:100A9F00017544907531107532B875460675472C3F
:100AAF00121F1690E67AE054FEF0E4FD7F90121BC1
:100ABF00497F647E001218DF7DFF7F42121B497F42
:100ACF00647E001218DF7D807F4E121B497535FF43
:100ADF0075388290E782E535F090E781E538F012BE
:050AEF001F29D2832243
:10176300121E9090E678E04480F07491121CBA90B7
:10177300E679E090E7C0121CBD90E679E090E7C1FE
:10178300121CBD90E679E090E7C2121CBD90E67989
:10179300E090E7C3121CBD90E678E04440121CBD04
:1017A30090E678E04480F07442121CBA90E679E542
:1017B30035121CBD90E678E04440121CBD90E678DB
:1017C300E04480F090E679744E121CBD90E679E512
:1017D30038121CBD90E678E04440121CBD021F295C
:1014A400E54B2401F54BE4354AF54AE43549F54961
:1014B400E43548F548E47FE87E03FDFCAB4BAA4ADB
:1014C400A949A848C31209AE7006FD7F90121B49B2
:1014D4007FA07E867D017C00AB4BAA4AA949A8481F
:1014E400C31209AE7009121E90121763121F297FCE
:1014F400407E0D7D037C00AB4BAA4AA949A848D382
:101504001209AE4009E4F54BF54AF549F5483004B3
:1015140020E533B401031210B8E533B40203121802
:101524008FE533B4040312183BE533B4630312129A
:04153400B5C2042216
:021F2C00D322BE
:021F2E00D322BC
:021F3000D322BA
:101A2F0090E680E030E71800000090E6207402F0A6
:101A3F00000000E490E621F0000000D205801600BF
:101A4F000000E490E620F000000090E6217440F0E2
:0D1A5F00000000C20590E6BAE0F541D32278
:101E350090E740E541F0E490E68AF090E68B04F007
:021E4500D322A6
:081F0E0090E6BAE0F527D322AA
:101E470090E740E527F0E490E68AF090E68B04F00F
:021E5700D32294
:021F3200D322B8
:021F3400D322B6
:021F3600D322B4
:10008000E4F518F51990E6B9E0244B60711470039B
:100090000202AF24F470030202E524FD70030203A0
:1000A0002F14700302039324FD70030203C814701D
:1000B000030204492417600302045BE490E68AF01B
:1000C00090E68BF090E6A0E020E1F990E68BE0F579
:1000D00018E4F5B5F5B390E60174CAF0E490E6C310
:1000E000F090E6C2F0D20400000090E6047480F0C4
:1000F0000000007402F0000000E4F002045DE490EF
:10010000E68AF090E68BF090E6A0E020E1F990E638
:100110008BE0F518D3943F4024E4F5197440251979
:10012000F582E434E7F583E0FF74AB2519F582E44A
:100130003427F583EFF00519E519B440DF9027AEB9
:10014000E0FFE4FCFDFEFB7A01F9F8120891C0041F
:10015000C005C006C0079027ADE0FFE4FCFDFEFB34
:10016000FA7901F8120891D003D002D001D000EF43
:100170002BFBEE3AFAED39F9EC38F89027AFE0FFB7
:10018000E4FCFDFEEB2FF53EEE3AF53DED39F53C96
:10019000EC38F53B9027ADE0F52CA3E0F52EA3E07D
:1001A000F52D7F9A121EC69027ABE0FF7E00121E2F
:1001B000CF9027ABE0FF7E00121ED89027ABE0FF68
:1001C0007E00121EE19027ACE075F004A4FFAEF0B3
:1001D000121EEA9027ACE075F004A4FFAEF0121EE8
:1001E000F39027ACE075F004A4FFAEF0121EFC9073
:1001F00027B0E0C3940250139027CCE090E6C07083
:1002000005744EF08016749CF080119027CCE0901D
:10021000E6C07005749FF08003749DF09027CEE0D7
:10022000F5399027CBE0F5379027CFE0F5429027BE
:10023000D9E0F536A3E0FEA3E07C002400F526EC2F
:100240003EF5259027B1E0F533E5337003753301B2
:100250009027B6E0FEA3E07C002400F529EC3EF5F3
:1002600028A3E0FEA3E02400F544EC3EF5439027EC
:10027000B2E0FEA3E02400F532EC3EF531A3E0FE4F
:10028000A3E02400F547EC3EF5469027BCE0FEA332
:10029000E02400F540EC3EF53F9027BAE0FEA3E0F5
:1002A0002400F530EC3EF52FE4FD7F900203C2E41C
:1002B000F51974AB2519F582E43427F583E0FF7452
:1002C000402519F582E434E7F583EFF00519E519C7
:1002D000B440DF000000E490E68AF000000090E601
:1002E0008B7440804390E74074ABF0A37408F0A394
:1002F000740AF0A37498F0A3740FF0A3747CF0A3B5
:100300007401F0A304F0A37493F0300505E4A3F0A6
:10031000800690E74974FFF0000000E490E68AF060
:1003200000000090E68B740AF0121C8F02045D90AE
:10033000E678E04480F090E6797491F07F647E0086
:10034000120EFF90E679E090E740F07F647E0012A5
:100350000EFF90E679E090E741F07F647E00120E98
:10036000FF90E679E090E742F07F647E00120EFF96
:1003700090E679E090E743F090E678E04440F000C2
:100380000000E490E68AF000000090E68B7404F030
:1003900002045DE490E68AF090E68BF090E6A0E03F
:1003A00020E1F990E68BE0F518D3940150030204A4
:1003B0005D90E741E0FD7F42121B4990E740E0FD80
:1003C0007F4E121B4902045DE490E68AF090E68BB2
:1003D000F090E6A0E020E1F990E68BE0F518D394E8
:1003E00001407A90E740E05480C413131354012471
:1003F000FF92A3E05440C41313540324FF92A2E0DD
:100400005420C413540724FF92A1E05410C4540F85
:1004100024FF92A0A3E075F00AA4FFAEF01218DF4B
:1004200090E740E05408131313541F24FF92A3E0F5
:1004300054041313543F24FF92A2E05402C3132424
:10044000FF92A1E01392A08014D2867F647E0012F6
:0E04500018DFC2867F647E001218DFD322C33D
:01045E00227B
:101DAE00C0E0C083C082D2015391EF90E65D740112
:081DBE00F0D082D083D0E032A6
:101DDE00C0E0C083C0825391EF90E65D7404F0D0F2
:061DEE0082D083D0E03238
:101DF400C0E0C083C0825391EF90E65D7402F0D0DE
:061E040082D083D0E03221
:101AA900C0E0C083C08285585485595585558285C3
:101AB9005483A37402F08550568551578557828502
:101AC9005683A37407F05391EF90E65D7410F0D03C
:061AD90082D083D0E03250
:101DC600C0E0C083C082D2035391EF90E65D7408F1
:081DD600F0D082D083D0E0328E
:101A6C00C0E0C083C08290E680E030E7208550540F
:101A7C00855155855582855483A37402F08558563B
:101A8C00855957855782855683A37407F05391EF78
:0D1A9C0090E65D7420F0D082D083D0E0325F
:010FFF0032BF
:011F38003276
:011F39003275
:011F3A003274
:1017E300C0E0C0F0C083C082C0D075D000C000C0CC
:1017F30001C002C003C004C005C006C007C2AF12C7
:101803001E9000000090E68F7404F00000005391D6
:10181300EF90E65FE04404F0121F29D2AFD007D067
:1018230006D005D004D003D002D001D000D0D0D050
:0818330082D083D0F0D0E03236
:10135A00C0E0C083C082C0D075D000C004C006C03F
:01136A00077B
:10136B00C2AF90E6A1E020E1F990E780E0146014B1
:10137B0024F8601E240C604624FE604614704875E9
:10138B002200804390E782E0F53590E781E0F53865
:10139B008035D28C90E781E0540FF534A3E0FEA3A7
:1013AB00E07C002400FFEC3EC313F52AEF13F52B72
:1013BB00754F00754E00754D00754C008009C28C41
:1013CB008005752200D20600000090E68DE4F053F4
:0B13DB0091EF90E65FE04408F0D2AF15
:0F13E600D007D006D004D0D0D082D083D0E03250
:011F3B003273
:011F3C003272
:011F3D003271
:011F3E003270
:011F3F00326F
:011F4000326E
:011F4100326D
:011F4200326C
:011F4300326B
:011F4400326A
:011F45003269
:011F46003268
:011F47003267
:011F48003266
:011F49003265
:011F4A003264
:011F4B003263
:011F4C003262
:011F4D003261
:011F4E003260
:011F4F00325F
:011F5000325E
:011F5100325D
:011F5200325C
:011F5300325B
:011F5400325A
:011F55003259
:011F56003258
:011F57003257
:011F58003256
:060BFC008F1A8C1B8D1CFA
:100C0200531A0753A0BF7F0A7E00120EFFE4F51DA0
:100C1200F51EC37402951EFFE51AA807088002C3D9
:100C220013D8FC30E00543A020800353A0DF7F0AE5
:100C32007E00120EFF43A0107F0A7E00120EFF53A9
:100C4200A0EF7F0A7E00120EFF051EE51E70020550
:100C52001DC39403E51D6480948040B6E4F51DF540
:100C62001EC37409951EFFE51CAE1BA8070880056C
:100C7200CEC313CE13D8F930E00543A0208003532E
:100C8200A0DF7F0A7E00120EFF43A0107F0A7E00C3
:100C9200120EFF53A0EF7F0A7E00120EFF051EE523
:100CA2001E7002051DC3940AE51D6480948040B144
:100CB20043A0407F0A7E00120EFF53A0BF7F0A7E30
:040CC20000020EFF1F
:091EC600AD07AC06E4FF020BFCC1
:091ECF00AD07AC067F04020BFC18
:091ED800AD07AC067F05020BFC0E
:091EE100AD07AC067F06020BFC04
:091EEA00AD07AC067F01020BFC00
:091EF300AD07AC067F02020BFCF6
:091EFC00AD07AC067F03020BFCEC
:101B49008D1AAD0790E678E04480F090E679EDF0E3
:101B59007F647E00120EFF90E679E51AF07F647EBD
:101B690000120EFF90E678E04440F07F647E0002A8
:021B79000EFF5D
:100E5500121E7B5380FE7F017E00120EFF121E7153
:100E65007F027E00120EFF121EBC7F027E00120E54
:100E7500FF121E9A7F027E00120EFF121F0A7F02CA
:100E85007E00120EFF121E607F027E00120EFF1200
:100E950019A27F027E00120EFF1213FC7F027E0054
:100EA500120EFF121E317F027E00120EFF121E71FE
:100EB5007F027E00120EFF121EBC7F027E00120E04
:100EC500FF121E9A7F027E00120EFF121F0A7F027A
:100ED5007E00120EFF121E607F027E00120EFF12B0
:100EE50019A27F027E00120EFF1213FC7F027E0004
:0A0EF500120EFF121E317F027E0074
:100EFF00EF7803C333CE33CED8F9FFEF4E6007EF51
:070F0F001F70F81E80F5229F
:0713F5007F037E00120EFFD2
:0413FC0053B1F722D0
:051F05007E00120EFF3A
:041F0A0043B10822B5
:071E93007F037E00120EFF29
:041E9A0053B17F229F
:101E2000121F29C206752201121F0A121EBC1219A6
:011E3000A20F
:041E310043B1802217
:0A1EA80053B1EF53B1BF53B1DF2275
:0A1EB20053B1FE53B1FB53B1FD2202
:071E59007F037E00120EFF63
:0A1E600053B1EF43B14043B120221B
:071E6A007F037E00120EFF52
:0A1E710053B1FE43B10443B1022255
:0A1EBC0043B11043B14043B12022AE
:101969007F017E00120EFF121E717F017E00120E92
:10197900FF121EBC7F017E00120EFF121E9A7F010C
:101989007E00120EFF121F0A7F017E00120EFF1247
:091999001E607F017E00120EFFAA
:0A19A20043B10143B10443B1022236
:0C1E7B00121E601213FC1219A2021E318C
:1019EE00121E7B7F0A7E00120EFF121EBC121E718B
:1019FE007F037E00120EFF121EB27F0D121F051204
:101A0E001E93121E6A121E597F0312199D1213F590
:101A1E007F037E00120EFF121E317F147E00020E17
:011A2E00FFB8
:1015C800E4FFFEE53CFDE4FCFB7A01F9F812091C96
:1015D800E4FB7A01F9F812091C8F2CE4FFE53DFEC3
:1015E800E4FDFCFB7A01F9F812091C8F2EE53EFF99
:0815F8008F2D1219AC1219EE3F
:10160000121E7B7F0A121F05121E9A7F037E001294
:101610000EFF121EA87F0D7E00120EFF121E311249
:1016200013F5121E59121E6A7F037E00120EFF125E
:101630001EBC121E937F03121F05121E597F031238
:10164000199D1213F57F037E00120EFF121E317FCB
:06165000147E00020EFFF3
:101C64005380FE1219697F011213F77F017E00125F
:101C74000EFF121E31C283121D5AD283121D5A1234
:0B1C840019697F01120EE94380012264
:071F1E00120E554380012261
:101E0A00120E55C283121D5AD283121D5A7F021214
:061E1A000E5D4380012271
:10192500121E7B120EFBE4FDFC1219707F011213CF
:10193500F77F017E00120EFF121E311219697F0119
:101945001213F77F017E00120EFF121E317F017EFA
:1019550000120EFF0DBD00010CED64927003EC64E6
:031965000470C645
:01196800225C
:1019AC00C2857F057E00120EFFD2857F057E001258
:1019BC000EFFC2857F057E00120EFFD2857F057E4D
:1019CC0000120EFFC2857F057E00120EFFD2857FAE
:1019DC00057E00120EFFC2857F057E00120EFFD21F
:0219EC00852252
:101C8F00E4F51AF51BD2827F1E7E001218DFC28286
:101C9F007F1E7E001218DF051BE51B7002051AC39D
:0A1CAF009405E51A6480948040DB80
:011CB9002208
:091E87001219251219EE121600C1
:031E9000C28222E9
:031F2900D282223F
:011F59002265
:011F5A002264
:101538001215C8E537B40102C287121F59E5397080
:101548006EE52C75F040A485F01AF51BAF227E00DD
:10155800AC1AAD1B12087FD3EF9400EE6480948020
:1015680040147FC47E03121CC2121763E51B151BAF
:1015780070DA151A80D6751A00852E1BAF227E00E8
:10158800AC1AAD1B12087FD3EF9400EE64809480F0
:1015980040147FC47E00121CC2121763E51B151B82
:1015A80070DA151A80D6AF2D7E00121CC28006E5AF
:0F15B80022640160FA121F5AE537B40102D2878C
:0115C7002201
:100D8F001215C8E537B40102C287121F599027CC3C
:100D9F00E07027F51CF51D7FA67E04121CC21217EA
:100DAF0063051DE51D7002051CC3940AE51C6480D4
:100DBF00948040E37FE67E0180047F807E0B121CCF
:100DCF00C2121600121F0AE539706AE52C75F04041
:100DDF00A485F01AF51BAF227E00AC1AAD1B1208CA
:100DEF007FD3EF9400EE940040147FC47E03121C57
:100DFF00C2121763E51B151B70DC151A80D8751A04
:100E0F0000852E1BAF227E00AC1AAD1B12087FD3BC
:100E1F00EF9400EE940040147FC47E00121CC212A7
:100E2F001763E51B151B70DC151A80D8AF2D7E00DC
:100E3F00121CC28006E522640160FA121F5AE537C0
:050E4F00B40102D2878E
:010E5400227B
:041BAD00AF40AE3F58
:101BB100AD07AC06D3ED9400EC9400401E0000008C
:101BC100EE90E6D0F0000000ED90E6D1F0000000CC
:0C1BD10075BB04000000E5BB30E7FB2200
:101D7900E542700C121538E530452F700F02192510
:0D1D8900E530452F70031219251215382280
:1010B8009027AEE0FFE4FCFDFEFB7A01F9F8120888
:1010C80091C004C005C006C0079027ADE0FFE4FC4E
:1010D800FDFEFBFA7901F8120891D003D002D00185
:1010E800D000EF2BFBEE3AFAED39F9EC38F89027FF
:1010F800AFE0FFE4FCFDFEEB2FF53EEE3AF53DEDEB
:1011080039F53CEC38F53B9027CCE0701E7FBA7E71
:1011180032AB3EAA3DA93CA83BD31209AE403CE500
:101128003E2446F53EE53D34CD801FE47F807E0BAE
:10113800FDFCAB3EAA3DA93CA83BD31209AE401B1F
:10114800E53E2480F53EE53D34F4F53DE53C34FFCD
:0F115800F53CE53B34FFF53B0216E21212102284
:1016E200121E20120D8F1219251219EE200671E515
:1016F20036D394004003121CE4D3E5269400E5257A
:1017020094004003120FD2E4F518F519C283121D9A
:101712000DD283121D0D121C640519E51970020504
:1017220018C39492E5186480948440E0121925123B
:101732001600E4F518F519C283121D0DD283121D8D
:101742000D121C640519E51970020518C39492E57F
:10175200186480948440E0121E28121BAD121E9061
:011762002264
:10121000121E20D286121538D2861219251219EE06
:101220003006030212B4E536D394004003121CE4E6
:10123000D3E5269400E52594004003120FD2E4F58F
:1012400018F519C283121D0DD283121D0D121C64D4
:101250000519E51970020518C39492E51864809485
:101260008440E0121F0A121EBC121E71121E31D2DF
:1012700086121538D286121925121600E536D39437
:10128000004003121CE4E4F518F519C283121D0D89
:10129000D283121D0D121C640519E5197002051880
:1012A000C39492E5186480948440E0121E28121BB7
:0412B000AD121E90CD
:0112B4002217
:10188F00121E20121538121E87200643E536D394F8
:10189F00004003121CE4D3E5269400E52594004094
:1018AF0003120FD2E4F518F519C283121D0DD2835E
:1018BF00121D0D121C640519E51970020518C39449
:0F18CF0092E5186480948440E0121E28121BAD2D
:0118DE0022E7
:10183B00121E20D286121538D286121E872006431E
:10184B00E536D394004003121CE4D3E5269400E55F
:10185B002594004003120FD2E4F518F519C2831238
:10186B001D0DD283121D0D121E0A0519E5197002EA
:10187B000518C39449E5186480948240E0121E2831
:03188B00121BAD80
:01188E002237
:1012B500121E20121538121E87300603021359E438
:1012C500F518F519121C640519E51970020518C3FE
:1012D5009404E5186480948040EAE4F518F519C390
:1012E500E5199529E5189528500D121C640519E591
:1012F5001970EC051880E8E536D394004003121CFC
:10130500E4D3E5269400E52594004003120FD2E4CA
:10131500F518F519C3E5199547E51895465012D204
:1013250083121D0D121C640519E51970E705188057
:10133500E3E4F518F519C3E5199544E51895435007
:101345000D121C640519E51970EC051880E8121ECC
:0413550028121BAD92
:011359002271
:101D0D00000000E53225E0E5313390E6D0F000002B
:101D1D0000E53225E090E6D1F000000075BB04002F
:081D2D000000E5BB30E7FB22DA
:101D5A00000000E490E6D0F000000090E6D104F024
:0F1D6A0000000075BB06000000E5BB30E7FB2260
:0B1CE400AF367E00AC31AD3212087F3D
:101CEF00AC06EC90E6D0F0000000EF90E6D1F000EB
:0E1CFF00000075BB06000000E5BB30E7FB22CD
:040FD200AF26AE2573
:100FD600AD07AC06000000ED25E0EC3390E6D0F05E
:100FE600000000ED25E090E6D1F000000075BB049E
:090FF600000000E5BB30E7FB221E
:081F1600E4F563D2E9D2AF2229
:101ADF0090E678E020E6F9C2E990E678E04480F0FD
:101AEF00EF25E090E679F090E678E030E0F990E6C7
:101AFF0078E04440F090E678E020E6F990E678E070
:061B0F0030E1D6D2E9220C
:101B7B00A90790E678E020E6F9E563702390E67814
:101B8B00E04480F0E925E090E679F08D5EAF03A9A3
:101B9B0007755F018A608961E4F562756301D32281
:021BAB00C32253
:101B1500A90790E678E020E6F9E563702590E67878
:101B2500E04480F0E925E0440190E679F08D5EAF70
:101B350003A907755F018A608961E4F5627563032E
:041B4500D322C322C2
:03004B00020AF4B2
:100AF400C0E0C083C082C085C084C086758600C043
:100B0400D075D000C000C001C002C003C006C00739
:100B140090E678E030E206756306020BDE90E67834
:100B2400E020E10CE56364026006756307020BDEF6
:100B3400E56324FE605F14603624FE7003020BCF6D
:100B440024FC7003020BDB24086003020BDEAB5FA2
:100B5400AA60A961AF6205628F82758300120830B2
:100B640090E679F0E562655E7070756305806B9060
:100B7400E679E0AB5FAA60A961AE628E82758300FC
:100B840012085D756302E55E6401704E90E678E0DC
:100B94004420F08045E55E24FEB5620790E678E0E7
:100BA4004420F0E55E14B5620A90E678E04440F033
:100BB40075630090E679E0AB5FAA60A961AE628ECE
:100BC4008275830012085D0562800F90E678E04428
:100BD40040F075630080037563005391DFD007D044
:100BE40006D003D002D001D000D0D0D086D084D09B
:080BF40085D082D083D0E032ED
:030000000216568F
:0C165600787FE4F6D8FD75816302169DD4
:10083000BB010CE58229F582E5833AF583E022507D
:1008400006E92582F8E622BBFE06E92582F8E222C7
:0D085000E58229F582E5833AF583E49322E1
:10085D00F8BB010DE58229F582E5833AF583E8F0D1
:10086D00225006E92582C8F622BBFE05E92582C87D
:02087D00F22265
:10087F00EF8DF0A4A8F0CF8CF0A428CE8DF0A42E8D
:02088F00FE2247
:10089100E88FF0A4CC8BF0A42CFCE98EF0A42CFC06
:1008A1008AF0EDA42CFCEA8EF0A4CDA8F08BF0A484
:1008B1002DCC3825F0FDE98FF0A42CCD35F0FCEBE3
:1008C1008EF0A4FEA9F0EB8FF0A4CFC5F02ECD39A8
:0F08D100FEE43CFCEAA42DCE35F0FDE43CFC2215
:1008E00075F008758200EF2FFFEE33FECD33CDCCCF
:1008F00033CCC58233C5829BED9AEC99E582984052
:100900000CF582EE9BFEED9AFDEC99FC0FD5F0D62E
:10091000E4CEFBE4CDFAE4CCF9A88222B800C1B958
:100920000059BA002DEC8BF084CFCECDFCE5F0CB96
:10093000F97818EF2FFFEE33FEED33FDEC33FCEBCF
:1009400033FB10D703994004EB99FB0FD8E5E4F98A
:10095000FA227818EF2FFFEE33FEED33FDEC33FC77
:10096000C933C910D7059BE99A4007EC9BFCE99A6B
:10097000F90FD8E0E4C9FAE4CCFB2275F010EF2FB0
:10098000FFEE33FEED33FDCC33CCC833C810D707B0
:100990009BEC9AE899400AED9BFDEC9AFCE899F8EB
:0E09A0000FD5F0DAE4CDFBE4CCFAE4C8F9227E
:1009AE00EB9FF5F0EA9E42F0E99D42F0E89C45F09F
:0109BE002216
:10166200020683E493A3F8E493A34003F68001F215
:1016720008DFF48029E493A3F85407240CC8C33389
:10168200C4540F4420C8834004F456800146F6DF58
:10169200E4800B0102040810204080900CC6E47E16
:1016A200019360BCA3FF543F30E509541FFEE4934D
:1016B200A360010ECF54C025E060A840B8E493A314
:1016C200FAE493A3F8E493A3C8C582C8CAC583CA3F
:1016D200F0A3C8C582C8CAC583CADFE9DEE780BEF7
:010D8E000064
:00000001FF
